:020000003328A3
:08000800CE000308CF00CF0871
:100010008300CE0E4E0E09000030860000308500B1
:100020008316F030850000308600FF308100831297
:100030000C3084008001840A50300406031D1A2805
:100040000800820700007E341434E634D6349C3431
:10005000DA34FA341634FE349E34403402346834D0
:10006000A8342A3400340C209021DF20B60BEF2076
:10007000DF20B60BA2203D203828902080202008C9
:10008000371D4528290874204928B71D49282A0802
:100090007420A80099209020AA0088202008371DED
:1000A0005428290874205828B71D58282A08742075
:1000B000A80099209020A900B820CF03CF0F9E2040
:1000C00088202008371D6728290874206B28B71D51
:1000D0006B282A087420A80099208A218A218A2165
:1000E0008A218A218A210800C800C900CC214A0837
:1000F000CC004B08CD00FF30CE00D6214F080800C1
:100100002F21903091004521403091004521080079
:100110002F21903091004521413091004521080068
:100120002F21913091004521121060213C211108AE
:1001300008002808910045213C2108009821AB21A6
:10014000EC2108003719AE28B719A928051537156D
:10015000B728051185113711B711B7280511851575
:100160003711B715B72885110515B71137150800D0
:10017000CF01A8010B30B100B2002908FE3C0318E2
:10018000C328A00108000A30B100B20029080A3CC7
:10019000031CCC28A0010800CF0A0800B003B00F50
:1001A000DB20320F212086008421310F21208600A0
:1001B0000614842108000B30B100B20008000130A1
:1001C000B600051A08008421842184218421051A9F
:1001D000EA28B60184218421051EEA2808006B3034
:1001E0008600B70184215630860084218020FF30AC
:1001F000910045213C21DF20B60BFF28EF28371561
:100200009020A800A1001921CE2080209920DF2075
:10021000B60B0B29FF283711B7159020A800A100B5
:100220001921CE2088209920B60BDF20B60B332869
:100230000B290A30B100B2001B30A10CA102031C33
:100240000800EC21210808002F2191309100452160
:1002500012102F2160213C211108A80008008501FF
:100260008316051000000000000085108312371966
:100270000515B71985150800831685148312851C8A
:100280003F29831605148312080008309000831656
:10029000910D05100318051485148312851C4E2931
:1002A00083168510900B4829000085148312851C45
:1002B000572912140518121083168510831208008E
:1002C0008316051408309000831685148312851C4C
:1002D0006729050C910D83168510900B652912185E
:1002E000051085148312851C732983168510080058
:1002F0000A30B30000000000000000000000000011
:100300000000B30B7A2908000A30B4007821B40B3E
:10031000862908001430B500CE20B50B8C290800C2
:100320000130B1000230B200CF00B701A0010800D7
:100330002A08C800C80AC80B9E29AA29FF30C9008C
:10034000CC214B08CD004A08CC002908CE00D6218C
:100350004F08A0000800FF302007CD00CC01031893
:10036000CC0A0310CD0DCC0D4D0898004C08990017
:100370000310CD0DCC0D0310CD0DCC0D1808CD07FD
:100380000318990A1908CC07FF30CE002008CE02C6
:10039000D6214F08A1000800CA01CB014B0849072C
:1003A0000318CA0ACB00C80BCE290800CE03CE0F13
:1003B000DC29FF30CF00EB29CF014E08CD02031C12
:1003C000E229E6290130CC02031CEB29CF0A031DE8
:1003D000DD29FF30CF0008000000C6016430A10213
:1003E000031CF4290D22EE294608B0006430A10751
:1003F000C6010A30A102031CFF290D22F929460873
:10040000B1000A30A107C6010130A102031C0A2A6B
:100410000D22042A4608B2000800C60A46080F3911
:0E042000093C0318162A4608063EC6000800CE
:02400E00FB3F76
:00000001FF
